:020000040000FA
:040000008FEF00F08E
:020008009AD08C
:08001800E8D00B6E960E036E9A
:10002000980E046E55D8D8B4CA90D8A4CA80FC0FD4
:10003000D8A0CA92D8B0CA82800E036E960E046E03
:10004000980E076E086ACAB025D8CAB223D842D81B
:100050000304CB6E03C005F004C006F00050096E27
:100060000A6E003C0A6A4BD808500B2E0AD0BE6EAE
:100070000C0EBD6E07BEBD8A07BCBD889394CA84B2
:100080001200BB6E0C0EBA6E07BEBA8A07BCBA88E5
:100090009492F5D700D8D890073204320332120078
:1000A000066A056EFF0E0526062200D0D8A01200B3
:1000B000030E046EE70E02D8F5D7046AFE0F036E36
:1000C000E86A045AD8A012000000030600D0F8D74E
:1000D000086A076A100EF36E0434073608360550B6
:1000E000075C0650085805E30550075E0650085A9D
:1000F000D88003360436F32EEFD703501200055094
:100100000902F3CF07F0F4CF08F006500902F350CC
:10011000082605500A02F350082607501200F86A14
:100120004F0EAF6E240EAC6E900EAB6E0001C69AF1
:10013000470E926EE00E936EC00E946E9DD09EAAF6
:100140001BD0060EAB1412E1E1CF28F0E2CF29F06C
:100150002A2A1EEE80F02A50E126000EE222AECFBF
:10016000E7FF28C0E1FF29C0E2FF1100AE50AE500A
:10017000AB98AB8811000AD0F2A408D0F2940E4AD2
:100180000F2A817A0D6AD6CF0CF0110011002A5087
:100190002B5C14E02B2AE9CF03F0EACF04F00EEE3B
:1001A00080F02B50E926000EEA22EF50036E03C0C8
:1001B000E9FF04C0EAFFD880120004D0E868036EAB
:1001C000D8A0120012002A6A2B6A9D8A9F8AF28E9A
:1001D000F28C12009D9A0EEE80F0000EEE6AE82E70
:1001E000FDD72A6A2B6A9D8A1200F29ED8CF5AFE4A
:1001F000E8CF5BFEE0CF5CFEE9CF5DFEEACF5EFEBE
:10020000E1CF5FFEE2CF60FED9CF61FEDACF62FEC2
:10021000F6CF63FEF7CF64FEF5CF65FEF3CF66FE43
:10022000F4CF67FEA6CF68FEF28E0001A192F29E87
:100230005ACED8FF5BCEE8FF5CCEE0FF5DCEE9FF93
:100240005ECEEAFF5FCEE1FF60CEE2FF61CED9FF76
:1002500062CEDAFF63CEF6FF64CEF7FF65CEF5FF20
:1002600066CEF3FF67CEF4FF68CEA6FFF28E1000D5
:100270009EA8FED7AD6E120094948B9494928B92AC
:10028000949A8B9A94988B98939A8A9A006A280EDB
:10029000056E260E066E020EC0DE226A5EEC03F0CC
:1002A000939A8A8A320EFCDE939A8A9A206A266A88
:1002B0008ADF90DFCD6AF294F28A870ED56EB16A3A
:1002C000A192A082D08EA292B00EB16E60DF106EAD
:1002D000BE0E105C07E3FE0E105C02E30BD102D0F1
:1002E000126A08D110AE21D0126A8D0E105C05E1A1
:1002F00010C012F01368146817D09D0E105C05E151
:1003000010C012F0156816680FD0AD0E105C05E134
:1003100010C012F01768186807D0BD0E105C04E119
:1003200010C012F019681A68E5D0125202E1E2D04A
:10033000E1D08D0E125C22E1132803E110C013F00E
:100340001BD010C014F0260E135C08E1006A280EC2
:10035000056E260E066E020E60DE0DD07A0E135C60
:1003600004E1269020908B9A06D07B0E135C03E16B
:10037000269220928B981368BDD0BCD09D0E125C43
:10038000D8A49FD0152803E110C015F098D010C054
:1003900016F016521AE1260E155C08E1006A280EC6
:1003A000056E260E066E020E38DE0DD07A0E155C36
:1003B00004E1269020908B9A06D07B0E155C03E119
:1003C000269220928B98156895D0260E155C09E12F
:1003D00016C000F0280E056E260E066E020E1DDEFB
:1003E0006DD07A0E155C34E18B8A26807F0E165C08
:1003F0002DE22080D6CF0CF0D7CF0DF000EE38F0F4
:10040000D8901634E926000EEA22EECF01F0EFCFA5
:1004100002F001C02CF002C02DF02CC001F02DC064
:1004200002F001500C241C6E02500D201D6E000EB7
:100430000E201E6E000E0F201F6E1EC030F01FC05B
:1004400031F01CC034F01DC035F001D0209036D002
:100450007B0E155C33E18B8826827F0E165C2DE2C5
:100460002082D6CF0CF0D7CF0DF000EE38F0D89028
:100470001634E926000EEA22EECF01F0EFCF02F0AB
:1004800001C02EF002C02FF02EC001F02FC002F0EC
:1004900001500C241C6E02500D201D6E000E0E200B
:1004A0001E6E000E0F201F6E1EC032F01FC033F0F4
:1004B0001CC036F01DC037F001D0209215681AD04C
:1004C00019D0AD0E125C0AE1172803E110C017F035
:1004D00003D010C018F049D80DD00CD0BD0E125C5E
:1004E00009E1192803E110C019F003D010C01AF077
:1004F0006FD800D0205238E020A01AD030C01EF0B3
:1005000031C01FF034C01CF035C01DF0D6CF0CF048
:10051000D7CF0DF01C500C5C1D500D581E500E58BE
:100520001F500F580F501F18D8B0800AD8B880D865
:1005300020A21AD032C01EF033C01FF036C01CF00B
:1005400037C01DF0D6CF0CF0D7CF0DF01C500C5C8F
:100550001D500D581E500E581F500F580F501F1889
:10056000D8B0800AD8B887D8B1D67A0E175C16E111
:1005700026A011D0208000EE38F0D8901834E9265B
:10058000000EEA22EECF01F0EFCF02F001C02CF016
:1005900002C02DF002D020908B9A18D07B0E175CF1
:1005A00015E126A211D0208200EE38F0D890183440
:1005B000E926000EEA22EECF01F0EFCF02F001C0F3
:1005C0002EF002C02FF002D020928B9817681200F4
:1005D000420E195C08E11A5203E122901AD802D0A7
:1005E00022808B8404D07B0E195CD8B402D81968A1
:1005F0001200006A280E056E260E066E020E0DEC25
:1006000000F020902092949A8B9A94988B98266A66
:100610001200006A280E056E260E066E020E0DEC04
:1006200000F08B94206A8B9A8B98266A276A1200B6
:1006300026B003D020908B9A1DD0D6CF0CF0D7CF08
:100640000DF02CC001F02DC002F001500C241C6EE6
:1006500002500D201D6E000E0E201E6E000E0F208B
:100660001F6E1EC030F01FC031F01CC034F01DC022
:1006700035F0827A120026B203D020928B981DD0DA
:10068000D6CF0CF0D7CF0DF02EC001F02FC002F066
:1006900001500C241C6E02500D201D6E000E0E2009
:1006A0001E6E000E0F201F6E1EC032F01FC033F0F2
:1006B0001CC036F01DC037F082781200F80E3A6E7A
:1006C000E90E3B6EFC0E3C6E740E3D6EFD0E3E6EF2
:1006D0004D0E3F6E7E0E406E3A0E416ECB0E426E58
:1006E0002E0E436E4468260E456E6D0E466E210E2C
:1006F000476E3F0E486E1D0E496E4A68190E4B6ECE
:10070000660E4C6E170E4D6E450E4E6E150E4F6EEC
:100710007F0E506E130E516E5268110E536EB60E50
:10072000546E100E556E990E566E0F0E576E9F0E2C
:10073000586E0E0E596EC30E5A6E0D0E5B6E5C6ACD
:100740005D6E500E5E6E0C0E5F6EB30E606E0B0E25
:10075000616E240E626E0B0E636EA30E646E0A0E43
:10076000656E2C0E666E0A0E676EC00E686E090E00
:10077000696E5C0E6A6E090E6B6E6C6A6D6EAA0E07
:100780006E6E080E6F6E5B0E706E080E716E110E3F
:10079000726E080E736ECD0E746E070E756E8C0E33
:1007A000766E070E776E500E786E070E796E170E06
:1007B0007A6E070E7B6EE20E7C6E060E7D6EAF0EBD
:1007C0007E6E060E7F6E800E806F060E816F530E5A
:1007D000826F060E836F280E846F060E856F866B00
:1007E000876FD90E886F050E896FB50E8A6F050E5B
:1007F0008B6F920E8C6F050E8D6F710E8E6F050EC6
:100800008F6F510E906F050E916F330E926F050E24
:10081000936F160E946F050E956FFA0E966F040E79
:10082000976FE00E986F040E996FC60E9A6F040EC4
:100830009B6FAE0E9C6F040E9D6F960E9E6F040E06
:100840009F6F800EA06F040EA16F6A0EA26F040E40
:10085000A36F550EA46F040EA56F410EA66F040E74
:10086000A76F2E0EA86F040EA96F1B0EAA6F040EA1
:10087000AB6F090EAC6F040EAD6FF70EAE6F030ECB
:10088000AF6FE60EB06F030EB16FD60EB26F030EF0
:10089000B36FC60EB46F030EB56FB70EB66F030E0F
:1008A000B76FA80EB86F030EB96F990EBA6F030E2B
:1008B000BB6F8C0EBC6F030EBD6F7E0EBE6F030E42
:1008C000BF6F710EC06F030EC16F640EC26F030E57
:1008D000C36F580EC46F030EC56F4C0EC66F030E68
:1008E000C76F400EC86F030EC96F340ECA6F030E78
:1008F000CB6F290ECC6F030ECD6F1F0ECE6F030E84
:10090000CF6F140ED06F030ED16F0A0ED26F030E8D
:10091000D36FD46BD56FF60ED66F020ED76FED0E78
:10092000D86F020ED96FE30EDA6F020EDB6FDA0EAC
:10093000DC6F020EDD6FD20EDE6F020EDF6FC90EAE
:10094000E06F020EE16FC10EE26F020EE36FB80EB0
:10095000E46F020EE56FB00EE66F020EE76FA90EB0
:10096000E86F020EE96FA10EEA6F020EEB6F9A0EAE
:10097000EC6F020EED6F920EEE6F020EEF6F8B0EAC
:10098000F06F020EF16F840EF26F020EF36F7D0EA8
:10099000F46F020EF56F760EF66F020EF76F700EA3
:1009A000F86F020EF96F690EFA6F020EFB6F630E9D
:1009B000FC6F020EFD6F5D0EFE6F020EFF6F570E95
:1009C0000101006F020E016F510E026F020E036FE4
:1009D0004B0E046F020E056F460E066F020E076F78
:1009E000400E086F020E096F3A0E0A6F020E0B6F6F
:1009F000350E0C6F020E0D6F300E0E6F020E0F6F64
:100A00002B0E106F020E116F260E126F020E136F57
:100A1000210E146F020E156F1C0E166F020E176F4B
:100A2000170E186F020E196F120E1A6F020E1B6F3F
:100A30000D0E1C6F020E1D6F090E1E6F020E1F6F32
:100A4000040E206F020E216F226B236FFC0E246FA9
:100A5000010E256FF70E266F010E276FF30E286F1C
:100A6000010E296FEF0E2A6F010E2B6FEB0E2C6F0C
:100A7000010E2D6FE70E2E6F010E2F6FE30E306FFC
:100A8000010E316FDF0E326F010E336FDB0E346FEC
:100A9000010E356FD80E366F010E376F0001120050
:020AA000FFD77E
:020000040030CA
:0300010006170ED1
:020005008580F4
:060008000FC00FE00F40E5
:00000001FF
